:020000040000FA
:0600000025280600120095
:08000800AC000E0EAE00010E6B
:10001000AD00AC0E2C0E08006830051C383083167D
:100020008100831208000130900010308B000730EF
:1000300099000800831600309F006830810003306B
:100040009500EF30850083120800132047211A2005
:10005000542059200C2081012F142E28FE308E00B0
:100060008B108B170E08031D3C28A80A92209B308A
:100070004F2107308E073228323C4F212E0EFC3E96
:10008000033E0318FA3EFD3EF420FC2075200C20B0
:100090000030A6070830A7070930A80792201430BF
:1000A0005B2192304F212E28FA306421FA306421EE
:1000B000080023303521203035217030352169305A
:1000C00035216330352150303521453035215430CC
:1000D00035213A3035212030352106302B212E3084
:1000E000352112302B218D200800230834212408CB
:1000F00034212E30352125083421260834212708C3
:10010000342128083421290834212A0834212B08D5
:100110003421203035212D0E2B210D3035210A3090
:1001200035210800B00128083007B001F63E031859
:10013000B00A031C0A3EA80027083007B001F63EAB
:100140000318B00A031C0A3EA70026083007B001B6
:10015000F63E0318B00A031C0A3EA6002508300725
:10016000B001F63E0318B00A031C0A3EA50024089D
:100170003007B001F63E0318B00A031C0A3EA40083
:1001800023083007B001F63E0318B00A031C0A3EEC
:10019000A30022083007B001F63E0318B00A031C82
:1001A0000A3EA20021083007B001F63E0318B00A4B
:1001B000031C0A3EA10020083007B001F63E0318D8
:1001C000B00A031C0A3EA00008000F3E4F21A00108
:1001D000A101A201A301A401A501A601A701A801F3
:1001E0000034752178210800851C2F142F18E52074
:1001F0002F1CF1202F100800B201B300B307031821
:10020000B20A3208B2073308B3070318B20A122140
:1002100034080F39A900350E0F39AA0035080F39F7
:10022000AB0008001030B100B401B5013330B407A1
:10023000B419F039B41B0F39B4023330B507B5190E
:10024000F039B51B0F39B502B30DB20DB50DB40DB4
:10025000B10B16290800B600360E2F2136080F39CB
:10026000F63E0318073E0A3E303EB7000310482111
:1002700074304F210830B800B70C482173304F213B
:10028000B80B3C2900000314482172304F29031495
:100290000030031C103A8519103A85000800F13E21
:1002A000B90039185329B9185529B9185729FC3EEE
:1002B000031857290800FF3EBA005E304F21603016
:1002C0004F21BA0B5F290800FF3EBB0063305B2162
:1002D0005D304F2163305B215F304F21BB0B6A29BA
:1002E000080075217621762175217621792100007B
:0402F0000000080002
:02400E00433F2E
:104200000600120000007700770077002E006C0097
:104210006500610070007300650063006F006E0050
:1042200064002E0063006F006D002F0070006900B5
:104230006300000043006F007000790072006900A5
:104240006700680074002000280063002900200037
:10425000320030003100390020004C006500610060
:1042600070005300650063006F006E0064002E0054
:1042700063006F006D002C00200041006C006C009A
:10428000200052006900670068007400730020007D
:1042900052006500730065007200760065006400DE
:0442A0002E000000EC
:00000001FF
